:030000000233CFF9
:0C33CF0078FFE4F6D8FD75814D0234163D
:10141C0020000A3C2E2E2E3E004950436F6E6E6506
:10142C0063745245510A004950436F6E6E65637484
:10143C00000A49504E6F41434B210A003E432C5643
:10144C002C43432CC0E4E0EFF2E5F020D1E8EDEAC8
:10145C00EEEC49500A003E432C4D41432C253032D2
:10146C0062583A25303262583A25303262583A2561
:10147C00303262583A25303262583A25303262584E
:10148C002C4D414320E0E4F0E5F10A003E432C569C
:10149C0045522C20332E3220EEF22025732025735A
:1014AC002CC2E5F0F1E8FF20495020ECEEE4F3EB20
:1014BC00FF0A004A756E203035203230313200314F
:1014CC00363A34313A3234003E432C4C442C505290
:1014DC004F473A2020202020202020202020202090
:1014EC0020202020202020202020202020202020F0
:1014FC0020202020202020202020202020202020E0
:10150C0020202020202020202020202020202020CF
:10151C0020202020202020202CC4E0F2E020EFF01E
:10152C00EEF8E8E2EAE828F4E0E9EB290A003E2AC2
:10153C002C312CCEF1EDEEE2EDFBE520EFE0F0E00E
:10154C00ECE5F2F0FB20F1E5F2E5E2EEE3EE20E86B
:10155C00EDF2E5F0F4E5E9F1E00A003E412C413012
:10156C00312C2562752E2562752E2562752E25620D
:10157C00752C495020E0E4F0E5F120E0E4E0EFF2D6
:10158C00E5F0E00A003E412C4130322C2562752EEC
:10159C002562752E2562752E2562752C495020E02A
:1015AC00E4F0E5F120EEF1ED2E20F1E5F0E2E5F0CE
:1015BC00E00A003E412C4130332C2562752E256209
:1015CC00752E2562752E2562752C495020E0E4F0AD
:1015DC00E5F120F0E5E72E20F1E5F0E2E5F0E00A98
:1015EC00003E412C4130342C2562752E2562752E1F
:1015FC002562752E2562752CCCE0F1EAE020F1E530
:10160C00F2E80A003E412C4130352C2562752E251E
:10161C0062752E2562752E2562752CD8EBFEE70AB5
:10162C00003E2A2C312CC4EEEF2E20EFE0F0E0EC43
:10163C00E5F2F0FB20F1E5F2E5E2EEE3EE20E8ED79
:10164C00F2E5F0F4E5E9F1E00A003E422C533031CA
:10165C002C2562752CC6E4E0F2FC20E7E0EFF0EEFE
:10166C00F1E020F1EEE5E4E8EDE5EDE8FF20EEF247
:10167C0020F1E5F0E2E5F0E00A003E422C53303276
:10168C002C2562752CCEE1ECE5ED20F120F1E5F096
:10169C00E2E5F0EEEC20E1E5E720EAE2E8F2E0ED4D
:1016AC00F6E8E90A003E422C5330332C2562752CA7
:1016BC00CFE5F0E5E7E0EFF3F1EA20EFF0E820EF1B
:1016CC00EEF2E5F0E520F1E2FFE7E820F120F1E5AC
:1016DC00F0E2E5F0EEEC0A003E422C5330382C25BB
:1016EC0062752CCCE5E4EBE5EDEDFBE920495020EF
:1016FC00EAE0EDE0EB28E7E0E4E5F0E6EAE020E400
:10170C00EE203520F1E5EA290A003E454E440A0058
:10171C000A44756D70582020202020303020303144
:10172C0020303220303320303420303520303620F9
:10173C0030372030382030392030412030422030B2
:10174C0043203044203045203046000A3A003A20ED
:10175C00000A000A44756D7044202020202030308F
:10176C0020303120303220303320303420303520BE
:10177C00303620303720303820303920304120307E
:10178C004220304320304420304520304600457202
:10179C0072206B657900526420656570726F6D0AFA
:1017AC00005264204D454D0A00526420436F64651D
:1017BC000A00577269746520436F64650A004465BA
:1017CC006275674950204F4E0A004465627567493F
:1017DC0050204F46460A0044656275675573657222
:1017EC00204F6E0A00446562756755736572204F11
:1017FC0046460A0044656275674D7367204F6E0A52
:10180C000044656275674D7367204F46460A004376
:10181C006F6E666967206C6F636B210A00577220CC
:10182C00656570726F6D0A00205361766520656581
:10183C0070726F6D210A00457272204D4143210078
:10184C004C6F61643E3E002A00CEF8E8E1EAE00A03
:10185C0000202D202575282575290A003C413031A2
:10186C003D003C4130323D003C4130333D003C4179
:10187C0030343D003C4130353D003C21003C533080
:10188C00313D003C5330323D003C5330333D003C45
:10189C005330353D003C5330383D003C5330363DE1
:0118AC00003B
:063B79000114000112001E
:103BC300C28E438910E4F58B758DB8D2ABD28E22A9
:03001B0002333F6E
:10333F00C0E0C083C082C0D0C28E758B00758DB8BF
:10334F00201E0675A61E75A6E10512D21AE5146099
:10335F000205140517E517540F7051E513D39401A7
:10336F0040021513D226E517543F7012D2189066FB
:10337F008EE0600A04F0E0D394B44002D21E90664F
:10338F0087E0600204F0906104E0600214F0906640
:10339F008FE0D394014003E014F0301D020515E5D2
:1033AF0016D394644004D21E80020516E511D394FF
:1033BF000140021511D28ED0D0D082D083D0E0320E
:1008DF00C291C290D2B5C2237D027C007F07123B2A
:1008EF005C8F27E527646060097D017F60123AF70E
:1008FF00D223E4FDFC7F0B123B5C8F27E52730E60C
:10090F00097D04E4FF123B1BD2237D017C007F078E
:10091F00123B5C8F27E5277008FD7FFF123AF7D255
:10092F0023302303126000C288C2A8C2AA758900AF
:10093F001236F790633FE0B4FA06A3E064CE607B13
:10094F00E4F52774372527F582E43463F583E4F063
:10095F000527E527B443EC90633F74FAF0A374CEF8
:10096F00F0A374CCF0906345740AF0E4A3F0A304F1
:10097F00F0A3F090633B74FFF0A3F0A3F0E4A3F0B7
:10098F009063567403F0E4F527E5272401FFE43361
:10099F00FE74372527F582E43463F583E0FD123AC0
:1009AF00D30527E527C3944340DFE4F5A775A61EBB
:1009BF0075A6E1907FF0F0A3F080FE90634A740378
:1009CF00F0A374CCF0E4906349F090668CF0A3F040
:1009DF00122DECC2B512329DC21E123916D223C28D
:1009EF0025C2249065777408F09062B57424F0E402
:1009FF00A3F090633FE09062B7F0906340E09062A5
:100A0F00B8F0906341E09062B9F0906342E0906279
:100A1F00BAF0906343E09062BBF0906344E0906261
:100A2F00BCF0751301E4906578F0C21FC220C2219B
:100A3F00C222202318AF27FE7D03122ED2E4FF120D
:100A4F00314A7E147F1CE4FBFDFC12290890668E50
:100A5F00E060037401F0E4906104F0F515906576A1
:100A6F00F0F516123BC375A70775A61E75A6E1D242
:100A7F00AFE4F516906104E0700312397090668F41
:100A8F00E06401701D9080007410F09080A874FFD6
:100A9F00F0A3F0A3F0A3F0E490668FF0D223C2246A
:100AAF00C225908008E0F52730E405D21F7410F0BE
:100ABF00E52730E508D2219080087420F0E5273033
:100ACF00E608D2209080087440F0E515C3940340E7
:100ADF0019908002E4F0908001F0908000F0E5150D
:100AEF0094064006E4F5151239169080A0E07003C5
:100AFF001237EF9080B8E070031237759080D0E016
:100B0F0070031238BA908000E07013301F10122A51
:100B1F000F906332EFF0D3940040031200269080C1
:100B2F0002E07006908000E06005D21D020A80C2CC
:100B3F001DE4F515906104E06003020A8020231282
:100B4F00906579E0600C7E147F1E122D04E4906591
:100B5F0079F030211212252A906332EFF0D39400EE
:100B6F004005E0FF12001F202003020D041223A3F3
:100B7F00906332EFF07003020A80906376E054BF07
:100B8F00247F7003020C5F147003020C3724026081
:100B9F0003020CA62023077E147F25122D04202785
:100BAF0003020D0490634EE07006906352E060679D
:100BBF00906683E0FF90634EE0B50724906684E073
:100BCF00FE90634FE0B50618906685E0FE90635087
:100BDF00E0B5060C906686E0FE906351E06E6037DC
:100BEF00906352E06F6003020D04906684E0FF9003
:100BFF006353E06F6003020D04906685E0FF90631E
:100C0F0054E06F6003020D04906686E0FF90635519
:100C1F00E06F6003020D04C21B9065787401F0123F
:100C2F000021751301020D0490668EE060037401BC
:100C3F00F090667BE0FF906378E06F6003020D0435
:100C4F0090667BE004F0E4F513906576F0020D04F6
:100C5F00301B03020D04906345E07003020A80907D
:100C6F0062B4E06008906356741EF080069063567D
:100C7F007403F0120020D21BE4F513906576F09008
:100C8F00668704F0E490667AF0A3F02023677E1461
:100C9F007F33122D04805E90668EE060037401F046
:100CAF00301B52906376E020E74B906378E0FF9023
:100CBF00667AE0FE6F600D906682E07007EE146F4B
:100CCF007033801390667AE004F0906332E0FFD3C4
:100CDF0094044003122C0F9060007482F0A37401EF
:100CEF00F0906378E0906002F07E607F007D0312E9
:100CFF0034E2020A80201B03020E27E513706E12E6
:100D0F002207EF60237E647F76906477E02404FDF2
:100D1F001234E2906682E07009906356E0F5130298
:100D2F000A80E4F513020A80906687E0D3943C4072
:100D3F003C906682E070369062B4E07030906687C7
:100D4F0004F012308EE4906476F0A37412F0906683
:100D5F007BE0906478F0A374FDF090610563A201CD
:100D6F0090647A63A2017F12121F558098123BD3B1
:100D7F008F27E527B401159060007483F0E4A3F08A
:100D8F007E607F007D021234E2020A80E527D39451
:100D9F0001401C9060007483F0A37401F0E52724D8
:100DAF00FEA3F07E607F007D031234E2020A80E52D
:100DBF001364016003020A80906576E004F020233B
:100DCF00077E147F3D122D04906576E0FFD39401CA
:100DDF00400B906356E0941E5003E004F0EFC39471
:100DEF0005400DC21BE4906578F0120021020A80C5
:100DFF007C667D8390634AE0FAA3E0FB7F021236A4
:100E0F00737E647F76906477E02404FD1234E29061
:100E1F006356E0F513020A80E51364016003020ACA
:100E2F0080906578E014604624FE604214700302DF
:100E3F000F1A24046003020A80E4F515202713908B
:100E4F0065787404F0906576E05401F07513010233
:100E5F000A809080027410F0E4906578F0906576C7
:100E6F0004F075131290668374FFF0020A80906687
:100E7F0083E07003020F049064767480F0906478BE
:100E8F007401F0E4A3F0A304F0A37430F0A3747B17
:100E9F00F0E4F527747D2527F582E43464F5837437
:100EAF007DF0747E2527F582E43464F583E4F0E564
:100EBF00272407906477F07C667D8390634AE0FA7D
:100ECF00A3E0FB7F021236737E647F76E527240949
:100EDF00FD1234E2906682E0601B120020D21BE408
:100EEF00F513906576F090668704F0E490667AF0DB
:100EFF00A3F0020A80302707E4906578F08006900F
:100F0F0065787404F0751312020A809080027410D1
:100F1F00F0751303906576E06401FFF090657874C7
:100F2F0001F0EF7019906352E06013FCA3E0FDA392
:100F3F00E0FEA3E0FF906683121D21020A809063FA
:100F4F004EE0FCA3E0FDA3E0FEA3E0FF906683125A
:070F5F001D21020A8080FE43
:010F66002268
:10002600906377E0B444047F0180027F009063769A
:10003600E0B447047E0180027E00EE5F604A906372
:100046003FE0906378F0906340E0906379F09063CE
:1000560041E090637AF0906342E090637BF09063B6
:1000660043E090637CF0906344E090637DF090639E
:10007600777452F09062AE63A2019080A863A201E9
:100086007F06121F550208D5906332E0C3940850CC
:10009600030208DE90633FE0FF906378E06F600341
:1000A6000208DE906340E0FF906379E06F60030230
:1000B60008DE906341E0FF90637AE06F6003020818
:1000C600DE906342E0FF90637BE06F60030208DE30
:1000D600906343E0FF90637CE06F60030208DE906C
:1000E6006344E0FF90637DE06F60030208DE906387
:1000F60077E06444701A9080A8E0B4FF139062AE73
:1001060063A2019080A863A2017F06121F5580108A
:100116009062B2E09080ACF09062B3E09080ADF077
:1001260090668EE060037401F090668F7464F090C0
:1001360063777452F0906376E0646D600302027830
:100146007BFF7A14794812190F7BFF7A1479629033
:10015600633FE0F530A3E0F531A3E0F532A3E0F527
:1001660033A3E0F534A3E0F53512190F7530FF75AA
:1001760031147532BF7533FF7534147535CB7BFF7B
:100186007A14799812190F7BFF7A1479D412190F01
:100196007BFF7A15793A12190F7BFF7A15796790EA
:1001A6006345E0F530A3E0F531A3E0F532A3E0F5D1
:1001B6003312190F7BFF7A15799190634EE0F53073
:1001C600A3E0F531A3E0F532A3E0F53312190F7B76
:1001D600FF7A1579BF906352E0F530A3E0F531A3BD
:1001E600E0F532A3E0F53312190F7BFF7A1579EDAE
:1001F60090633BE0F530A3E0F531A3E0F532A3E0F0
:10020600F53312190F7BFF7A167910906337E0F5F4
:1002160030A3E0F531A3E0F532A3E0F53312190F70
:100226007BFF7A16792D12190F7BFF7A167956A263
:1002360027E433F53012190F7BFF7A16798690661C
:1002460082E0F53012190F7BFF7A1679B190668E2F
:10025600E0F53012190F7BFF7A1679E49062B4E06C
:10026600F53012190F1231FA7BFF7A177916121927
:100276000F22906376E0644C70737E177F1CFBFD43
:10028600FC12290890637EE0F528A3E0F529E4F541
:100296002BE528906380F0A3E529F07E177F577C35
:1002A600637D807B02122908E4F52A852982852848
:1002B60083E0FF7480252AF582E43463F583EFF04A
:1002C6000529E52970020528052AE52AB410DC7EF1
:1002D600177F5A7C637D807B10122908052BE52B3E
:1002E600C3941040AC7E177F5D122D042290637676
:1002F600E0646C7060F52C7E177F5FFBFDFC1229B5
:1003060008E4F52BE4906380F0A3E52CF07E177FDC
:10031600577C637D807B02122908E4F52AA82CE627
:10032600FF7480252AF582E43463F583EFF0052C0B
:10033600052AE52AB410E67E177F5A7C637D807B0A
:1003460010122908052BE52BC3940840B77E177FAA
:100356005D122D0422906376E0644B7061F52A7479
:1003660068252AF582E43463F583E06032746825F3
:100376002AF582E43463F583E0F460237468252A61
:10038600F582E43463F583E0FF747E252AF582E482
:100396003463F583E0B50710052AE52AB408C09052
:1003A60061047432F00208D59063767421F030232C
:1003B600030208D57E177F9A122D040208D5906392
:1003C60076E0B4521A2023077E177FA2122D0490DE
:1003D60063767472F07E637F767D0812345B2290BA
:1003E6006376E0644970452023077E177FAD122DA2
:1003F6000490637EE0F528A3E0F529E4F52A852933
:1004060082852883E0FF7480252AF582E43463F52B
:1004160083EFF00529E52970020528052AE52AB4A7
:1004260080DC7E637F767D8A12345B22906376E081
:10043600644370462023077E177FB5122D04906310
:100446007EE0F528A3E0F529E4F52A8529828528AA
:1004560083E493FF7480252AF582E43463F583EF01
:10046600F00529E52970020528052AE52AB480DB6E
:100476007E637F767D8A12345B22906376E0645ACF
:1004860070532023077E177FBE122D0490637EE0F3
:10049600F528A3E0F5297C637D807B80AF29AE2813
:1004A600123A78E4F52A852982852883E493FF7435
:1004B60080252AF582E43463F583EFF00529E529E2
:1004C60070020528052AE52AB480DB7E637F767DE7
:1004D6008A12345B22906376E06444600302056C02
:1004E60090637EE0FF644470030208D5EFB4310CDC
:1004F600C2237E177FCA122D040208D590637EE0C0
:10050600B4300CD2237E177FD6122D040208D59064
:10051600637EE0B4320CD2247E177FE3122D0402F0
:1005260008D590637EE0B4330CC2247E177FF112A7
:100536002D040208D590637EE0B4340CD2257E18D3
:100546007F00122D040208D590637EE0B4350CC2FC
:10055600257E187F0D122D040208D590637EE0FFDC
:1005660012001E0208D5906104E070132023077E56
:10057600187F1B122D049063767421F00208D59023
:1005860061047432F0906376E0FFB45104C2AF8028
:10059600FEEF645770452023077E187F29122D042D
:1005A60090637FE0906332F0E4F52A906332E0FFD7
:1005B600E52AC39F40030208D57480252AF582E404
:1005C6003463F583E0FF90637EE0252A24ADF5824F
:1005D600E43461F583EFF0052A80D0906376E06419
:1005E60053600302068F2023077E187F34122D04E2
:1005F60090633FE0FF9061B6E06F703C906340E02F
:10060600FF9061B7E06F7030906341E0FF9061B892
:10061600E0B50724906342E0FF9061B9E0B50718A2
:10062600906343E0FF9061BAE0B5070C906344E045
:10063600FF9061BBE06F60169063767421F0302303
:10064600030208D57E187F43122D040208D5E4F56F
:100656002AE4F516AF2AFE74AD252AF582E4346144
:10066600F583E0FD123AD3052AE52AC394FE40E15C
:10067600C2AFE4907FF0F0A3F0907FFD74AAF0A3E0
:1006860074FFF0A37455F080FE906376E0644F70BB
:100696005A90637EE0F528A3E0F529E52945287000
:1006A6000A2023077E187F4C122D042023077E186C
:1006B6007F53122D04E4F52A7480252AF582E4344A
:1006C60063F583E0852982852883F00529E529706D
:1006D600020528052AE52AB480DE90668DE024808E
:1006E600F090668CE03400F00208D5906376E06402
:1006F60045707490637EE0FEA3E0FF907FF0EEF01D
:10070600A3EFF0D39400EE94044038907FF0E0FE1F
:10071600A3E0FF90668CE0FCA3E0FD9FEC9E4023E7
:10072600E42FFFEE3401FED3ED9FEC9E5015C2AFD1
:10073600907FFD74AAF0A374FFF0A37455F0E4F55E
:10074600A780FE7E187F55122D047BFF7A18795DEF
:10075600907FF0E0F530A3E0F53190668CE0F5325D
:10076600A3E0F53312190F906376E0646560030227
:1007760008DE90637EE0FFA3E0907FF0CFF0A3EF6A
:10078600F0E4F528F529D3907FF1E09529907FF0E4
:10079600E095284020E4F5162529FFE5283401FEDA
:1007A600852982852883E0FD123AD30529E529703B
:1007B60002052880D17E187F68123569EF4E6020C9
:1007C600120003906345EFF0120003906346EFF0CA
:1007D600120003906347EFF0120003906348EFF0B6
:1007E6007E187F6E123569EF4E602012000390630B
:1007F6004EEFF012000390634FEFF0120003906388
:1008060050EFF0120003906351EFF07E187F7412E0
:100816003569EF4E6020120003906352EFF012002C
:1008260003906353EFF0120003906354EFF012004D
:1008360003906355EFF07E187F7A123569EF4E60AC
:100846002012000390633BEFF012000390633CEF2D
:10085600F012000390633DEFF012000390633EEF49
:10086600F07E187F80123569EF4E602012000390EB
:100876006337EFF0120003906338EFF01200039035
:100886006339EFF012000390633AEFF0E4F52AE4DF
:10089600F516E52A2401FFE433FE7437252AF5828E
:1008A600E43463F583E0FD123AD3052AE52AC394BE
:1008B6004340DCC2AFE4907FF0F0A3F0907FFD747C
:1008C600AAF0A374FFF0A37455F0E4F5A780FE7EAA
:0808D600637F767D0812345B9C
:0108DE0022F7
:103A0A00AE07EEC39430400BEED394395005EE2442
:103A1A00D0FF22EEC39461400BEED394665005EEBC
:103A2A0024A9FF22EEC39441400BEED394465005DD
:083A3A00EE24C9FF22AF0622B1
:103B95009062ADE004F070069062ACE004F09062D3
:0A3BA500ACE0FEA3E0FF123B3F225C
:10000300123B95123A0AEFC454F0FEC006123B9518
:08001300123A0AD0E02FFF228F
:10385D00E49069C8F0123B959069C9EFF0C39430BC
:10386D004018E0FFD3943950119069C8E02405F554
:10387D0082E43461F583EFF080119069C8E024058E
:10388D00F582E43461F583E4F0800C9069C8E004BE
:10389D00F0E0D3940840BE752B00752C00752D00FB
:0C38AD00E4F52E7B017A6179051220639E
:0138B90022EC
:043569008E2D8F2EE6
:10356D009062ACE4F0A374FFF0123B95EF606EF443
:10357D00606B852E82852D83E493B507EC752F0145
:10358D00E52E252FF582E4352DF583E49360259006
:10359D0062ADE0252FFF9062ACE03400FE123B3FA0
:1035AD00E52E252FF582E4352DF583E493B507043B
:1035BD00052F80CCE52E252FF582E4352DF583E4FE
:1035CD009370A6E52F24FFFFE434FFFE9062ADE07B
:1035DD002FF09062ACE03EF07E007F0122E4FEFF12
:0135ED0022BB
:102DEC007E187F86123569EF4E70037F01227E18A4
:102DFC007F89123569EF4E600C123B95EF24D0247D
:102E0C00FF92278002D2277E187F8F123569EF4EF2
:102E1C00600C123B95EF24D0906682F08005E49014
:102E2C006682F07E187F95123569EF4E600C123B6E
:102E3C0095EF24D090668EF08005E490668EF07E3F
:102E4C00187F9B123569EF4E600C123B95EF24D026
:102E5C0024FF92198002C2197E187FA1123569EFE6
:102E6C004E600C123B95EF24D09062B4F08005E4D8
:102E7C009062B4F090633F63A20190667C63A20100
:102E8C007F06121F5530193B7E187FA7123569EF4C
:102E9C004E603012000390667CEFF01200039066D7
:102EAC007DEFF012000390667EEFF0120003906647
:102EBC007FEFF0120003906680EFF0120003906633
:062ECC0081EFF07F0022FF
:1039C100906577E0C3947C40027F0A906577E0FEC2
:1039D10004F074B52EF582E43462F583EFF0BF0A8A
:1039E10027906577E0FF04F074B52FF582E4346227
:1039F100F583E4F0906577E0FF1235EE906577741A
:093A010008F09062B6E004F02226
:100F67003E2A2C312CCFE0F0E0ECE5F2F0FB20E05C
:100F7700F1E8EDF5F0EEEDEDEEE3EE20EFEEF0F259
:100F8700E02E20D0E5E6E8EC20F0E0E1EEF2FB20F1
:100F97002D20EFE0EAE5F2EDFBE90A003E4C2C4993
:100FA70030312C256C752CD1EAEEF0EEF1F2FC20F5
:100FB700EEE1ECE5EDE02C35302C3130302C3330E0
:100FC700302C3630302C313230302C323430302C1B
:100FD700343830302C393630302C31393230302CEF
:100FE70033383430302C35373630302C31313532D8
:100FF70030300A003E422C4930322C2562752CD302
:10100700EFF0E0E2EBE5EDE8E520EFEEF2EEEAEEF9
:10101700EC20EFF0E820EFE5F0E5E4E0F7E5202845
:101027005254532D435453290A003E532C4930330D
:101037002C2562752CC7E0E4E5F0E6EAE020F1F242
:10104700E0F0F2E020EFE5F0E5E4E0F7E8282A3108
:1010570030ECF1290A003E422C4930342C256275C8
:101067002CD0E5E6E8EC20EFE5F0E5E4E0F7E82052
:101077003720E1E8F20A003E422C4930352C256240
:10108700752CCFE5F0E5E4E0F7E020F120EAEEED9E
:10109700F2F0EEEBFCEDFBEC20E1E8F2EEEC0A00FF
:1010A7003E422C4930362C2562752CCAEEEDF2F003
:1010B700EEEBFCEDFBE920E1E8F2202D20F7E5F26D
:1010C700EDEEF1F2FC0A003E422C415030372C2560
:1010D70062752CC6E4E0F2FC20EAE2E8F2E0EDF605
:1010E700E8FE20EEF220F3F1F2F0EEE9F1F2E2E0B1
:1010F7000A003E422C415030382C2562752CCAE23A
:10110700E8F2E8F0EEE2E0F2FC20EFE0EAE5F2FBDD
:1011170020EEF220F3F1F2F0EEE9F1F2E2E00A005C
:101127003C21003C4930313D003C4930323D003CD8
:101137004930333D003C4930343D003C4930353D72
:10114700003C4930363D003C415030373D003C4182
:101157005030383D000A53656E64204B56543A2090
:10116700202020000ACFF0E5E2FBF8E5EDE8E520D6
:10117700ECE0EAF12E20E4EBE8EDFB20EFE0EAE516
:10118700F2E020EDE020EEF2EFF0E0E2EAF32100FA
:101197000ACFE5F0E5EFEEEBEDE5EDE8E520E1F36D
:1011A700F4E5F0E020EDE020EEF2EFF0E0E2EAF324
:1011B70021000A546F4164643A2020202020202017
:1011C700000A53656E64205061636B65743A2000B2
:1011D7000A435243206572726F7221202020000A51
:1011E700CEF2E2E5F7E0FE20EDE020E7E0E3F0F302
:1011F700E7EAF321000A526563204B5654000A526E
:101207006563206F6B21202020202020005443504D
:10121700005544500000112332465765748C9DAF2A
:10122700BECADBE9F810013322564775649C8DBFAF
:10123700AEDACBF9E82130021367764455ADBC8EA0
:101247009FEBFAC8D93120120377665445BDAC9E8F
:101257008FFBEAD8C94253617004152736CEDFEDFC
:10126700FC8899ABBA5243716014053726DECFFD6F
:10127700EC9889BBAA6372405125340617EFFECC60
:10128700DDA9B88A9B7362504135241607FFEEDC4F
:10129700CDB9A89A8B8495A7B6C2D3E1F008192BCC
:1012A7003A4E5F6D7C9485B7A6D2C3F1E018093B2F
:1012B7002A5E4F7D6CA5B48697E3F2C0D129380A20
:1012C7001B6F7E4C5DB5A49687F3E2D0C139281A0F
:1012D7000B7F6E5C4DC6D7E5F48091A3B24A5B697C
:1012E700780C1D2F3ED6C7F5E49081B3A25A4B79EF
:1012F700681C0D3F2EE7F6C4D5A1B082936B7A48E0
:10130700592D3C0E1FF7E6D4C5B1A092837B6A58CE
:10131700493D2C1E0F0089129B24AD36BF48C15A88
:10132700D36CE57EF78108931AA52CB73EC940DB3D
:1013370052ED64FF76028B109926AF34BD4AC3582D
:10134700D16EE77CF5830A9118A72EB53CCB42D91D
:1013570050EF66FD74048D169F20A932BB4CC55E05
:10136700D768E17AF3850C971EA128B33ACD44DFFD
:1013770056E960FB72068F149D22AB30B94EC75CED
:10138700D56AE378F1870E951CA32AB138CF46DDDD
:1013970054EB62F97008811A932CA53EB740C952E5
:1013A700DB64ED76FF89009B12AD24BF36C148D3BD
:1013B7005AE56CF77E0A8318912EA73CB542CB50AD
:1013C700D966EF74FD8B029910AF26BD34C34AD19D
:1013D70058E76EF57C0C851E9728A13AB344CD5685
:1013E700DF60E972FB8D049F16A920BB32C54CD77D
:1013F7005EE168F37A0E871C952AA338B146CF546D
:10140700DD62EB70F98F069D14AB22B930C74ED55C
:051417005CE36AF178BE
:103B7F0052669000000000000000000000000000EE
:053B8F00000000000031
:103AAC0074B42549F582E43467F583EFF005499049
:103ABC0067AFE549F064646005E549B4E408D208F1
:073ACC006349805349802289
:01001E0022BF
:030023000227FAB7
:0B27FA00C0E0C083C082C0D075D018C2
:1028050020980302288A751401AE99200210BE0291
:1028150009D291754605D2028069C2918065300F53
:102825001EC20F301007AF1E123AAC8053AF4905D8
:102835004974B42FF582E43467F583EEF08041BE28
:102845000904D20F803ABE02055349808032BE0387
:10285500159067AFE549F0634980534980C202D2BC
:1028650008754600801A301007AF1E123AAC80106A
:10287500AF49054974B42FF582E43467F583EEF06A
:10288500754605C29830997030036B301107309743
:1028950004D20080619066A4E0FFE54AC39F401121
:1028A500C203D214C290200B02D216C20BD296805C
:1028B50045AF4A054A74B42FF582E43468F583E0E0
:1028C500F54B300919534B7F30012820D0082004DF
:1028D50022634B80801D30041A634B8080153001C4
:1028E50012E54B524B300406A2D0929B8005A2D034
:0A28F500B3929B854B99C299D2AFB4
:0928FF00D0D0D082D083D0E032A9
:1031FA007BFF7A0F796712190F9069B4E0FEA3E09A
:10320A00FFC3E49FFFE49EFEAB07FA3395E0F9F8AB
:10321A007F007E8C7D0A7C00121C708F338E328D6B
:10322A00318C307BFF7A0F79A312190F7BFF7A0F4B
:10323A0079FBA211E433F53012190F7BFF7A10796A
:10324A003185473012190F7BFF7A10795DA209E4A4
:10325A0033F53012190F7BFF7A10797EA201E4331D
:10326A00F53012190F7BFF7A1079A7A204E433F51F
:10327A003012190F7BFF7A1079CEA212E433F5309F
:10328A0012190F7BFF7A1079F9A20AE433F530128A
:03329A00190F22E7
:102B13007E117F27123569EF4E70037F01227E11EC
:102B23007F2A123569EF4E602312385DA804A90588
:102B3300AA06AB077F007E8C7D0A7C00121C7012F4
:102B43001D029069B4EEF0A3EFF0800A9069B474AB
:102B5300FFF0A374B8F07E117F30123569EF4E6039
:102B63000C123B95EF24D024FF92118002C2117EF8
:102B7300117F36123569EF4E600712385D8F47803B
:102B830003E4F5477E117F3C123569EF4E600C126A
:102B93003B95EF24D024FF92098002C2097E117F66
:102BA30042123569EF4E600C123B95EF24D024FF9F
:102BB30092018002C2017E117F48123569EF4E6097
:102BC3000C123B95EF24D024FF92048002C2047EB2
:102BD300117F4E123569EF4E600E123B95EF24D0F4
:102BE30024FF920592128004C205C2127E117F5502
:102BF300123569EF4E600E123B95EF24D024FF92FD
:0C2C030005920A8004C205C20A7F00226C
:10329D00C203C216C208C202C20FE4F54A9066A468
:1032AD00F0F549F514C200D297D2969067B0F0C2EE
:1032BD0006C2159066A27409F0A3F0C209C204C239
:1032CD0001C213C211E4F547F546D2149069B474E6
:1032DD00FFF0A374B8F0C20AC205C212122B1390EC
:1032ED0067A57401F0C2ADE4F5C9D2CDD2CCC2C987
:1032FD00C2CAF5CDF5CC9069B4E0F5CBA3E0F5CA23
:10330D0085CBCD85CACCE4F59830010C2009095345
:10331D0087BFD29FD29E8002D29E438740C29FC25A
:10332D00ACC298C29975B81075B710D2CAD29CD2DA
:02333D00AC22C0
:103BAF00E54D6FFF90131C93654CF54DEF90121C74
:033BBF0093F54C2F
:013BC20022E0
:01001F0022BE
:04269B008E2A8F2BC9
:10269F00E4F52CF54DF54CAA06A9077B018B308A82
:1026AF00318932121C22042532F532E43531F531ED
:1026BF0030050F9067A6E0AB30AA31A932121C2269
:1026CF00800D9066A3E0AB30AA31A932121C22759F
:1026DF003001852A31852B320D0DE4FEEEC39D505E
:1026EF0018AB300532E532AA317002053114F912F8
:1026FF001C09FF123BAF0E80E3AB300532E532AA67
:10270F00317002053114F9E54D121C22AB30AA319C
:10271F00A932E54C121C220D0D300E0F9067B1E05F
:10272F00A3E0FAA3E08A2EF52F8006752E68752F89
:10273F00B4753001852A31852B32852F82852E8302
:10274F007402F0052FE52F7002052E052CE4FEEE26
:10275F00C39D504EAB30AA31A932121C09F52D641E
:10276F0002600BE52D64036005E52DB40913852F79
:10277F0082852E837409F0052FE52F7002052E0533
:10278F002C852F82852E83E52DF0052FE52F7002E6
:10279F00052E052C74012532F532E43531F5310E55
:1027AF0080AD852F82852E837403F0052FE52F7062
:1027BF0002052E052C906696E0FCA3E0FDA3E0FE3B
:1027CF00A3E0FFE4FAF9F8EF2401FFEA3EFEE93D4A
:1027DF00FDE83CFC906696121D219067B17401F0E4
:0A27EF00A3E52EF0A3E52FF0AF2CB8
:0127F90022BD
:10308E00E4FF9066A3E0FE7D000FED2405F582E4DB
:10309E003461F583EEF00F74052401F582E434619A
:1030AE00F583E4F07C667D95FEED1DAA0470011C8F
:1030BE00F5828A83E0FBAA070F74052AF582E434B1
:1030CE0061F583EBF00EBE04E07C667D99E4FEEDC7
:1030DE001DAA0470011CF5828A83E0FBAA070F74F7
:1030EE00052AF582E43461F583EBF00EBE04E07C34
:1030FE00667D9DE4FEED1DAA0470011CF5828A8397
:10310E00E0FBAA070F74052AF582E43461F583EB20
:10311E00F00EBE04E07C667DA1E4FEED1DAA0470F7
:10312E00011CF5828A83E0FBAA070F74052AF5823B
:0B313E00E43461F583EBF00EBE04E00A
:013149002263
:073BEC00C299D299D2902288
:0100200022BD
:103A4200AD077E677FA512269B9066A4EFF0D20396
:103A5200E4F54A30250D7E117F5C7C687DB4E0FB85
:103A6200122908C296301103D20022E5476003F5FD
:063A72001122123BEC22C0
:022C0F008F280C
:102C1100E528D394FA4012202503022D037E117F6B
:102C21006BE4FBFDFC122908223003427A6979B377
:102C31007B01C003C002C0019067B1E0A3E0FAA329
:102C4100E07E002528F9EE3AFAC3D082D083D0E0A5
:102C5100E99582EA95834012202503022D037E1116
:102C61007F97E41BFDFC12290822C2ACD20E9063AF
:102C710079E09066A3F0300E177E637F78E5282413
:102C8100FCFD12269B8F299066A4E02529F0801176
:102C91007E637F78E52824FCFD12269B9066A4EFD5
:102CA100F0A21282055005754805D215D203200EF7
:102CB10017E4F54AC296301104D200800BE5476053
:102CC10004F5118003123BEC302531300E1E7E11CC
:102CD1007FB99067B1E0A3E0FAA3E0AC02C3952904
:102CE100FDEC9400FCAB2912290880107E117FC8ED
:102CF1007C687DB49066A4E0FB122908C20EC2165E
:022D0100D2AC52
:012D030022AD
:10220700200603300B037F002220080302239830A7
:1022170010037F0022C208C291E4906476F09067B1
:10222700AFE0FF547F24FCF528906477F090667B3D
:10223700E0906478F0EF5480FF24B5F582E43467CA
:10224700F583E0906479F074B42FF582E43467ADD8
:1022570082FCE4F54DF54CFE9067AFE0547FF9EE54
:10226700C39950140DEDAA0470010C14F5828A83EA
:10227700E0FF123BAF0E80E0E54C454D6044302552
:10228700197E117FD79067AFE0548024B4F582E4BC
:102297003467AD82FCAB0112290890669AE0FCA373
:1022A700E0FDA3E0FEA3E0FFE4FAF9F8EF2401FF65
:1022B700EA3EFEE93DFDE83CFC90669A121D2102CC
:1022C70023983005249067AFE05480FF24B4F5824B
:1022D700E43467F583E09067A5F074B52FF582E4E1
:1022E7003467F583E09067A6F0E5287039C215F5E5
:1022F700489067A6E0B4E01E7490F020050302231F
:1023070098D2062025030223987E117FE6E4FBFD81
:10231700FC122908807B3025787E117FFCE4FBFDC9
:10232700FC122908806B9067AFE0548024B6F582D1
:10233700E43467F58363A20190647A63A201AF284E
:10234700121F5530251C7E127F059067AFE0FB54A6
:102357008024B4F582E43467AD82FCEB547FFB1232
:102367002908906692E0FCA3E0FDA3E0FEA3E0FF4E
:10237700E4FAF9F8EF2401FFEA3EFEE93DFDE83C07
:10238700FC906692121D21A20A82055002D206D243
:0B23970017301705C2177F01227F00DE
:0123A2002218
:0100210022BC
:10397000300008209705C200123BECE511B40106A7
:10398000E4F511123BEC302625C226E546600DD544
:10399000460A634980534980C202C29130120FE542
:1039A00048600BD54808E4F54AD203754805A20AD9
:1039B0008206500C200309E4FF123A42C206D20BE1
:0139C00022E4
:0E3BD300301608201505C2167F01227F002241
:103916009080007480F090633763A201F583F5828E
:1039260063A2017F08121F5590633F63A201908036
:103936008863A2017F0A121F559080927407F0A334
:1039460074D0F0A37406F0906349E0FF9080B1F064
:103956009080E1EFF09080957455F0A3F090800090
:0A3966007401F090800974F0F02263
:1037EF00908009E04410F09080A0E070609080A17C
:1037FF007482F09080A874FFF0A3F0A3F0A3F07F81
:10380F00039080AEEFF0A374CBF09080007402F0C1
:10381F009069BA121D2D000000009069BAE09080E7
:10382F0040F09069BBE0908041F09069BCE09080DF
:10383F0042F09069BDE0908043F0A3E4F0A3F0A3C1
:0D384F00F0A3F0908018F0A3F0A3F0A3F018
:01385C002249
:1038BA00908009E04440F09080D17482F07F0390B8
:1038CA0080DEEFF0A374CCF09080027402F090696D
:1038DA00BE121D2D000000009069BEE0908058F0D5
:1038EA009069BFE0908059F09069C0E090805AF0EA
:1038FA009069C1E090805BF0A3E4F0A3F0A3F0A389
:0B390A00F0908030F0A3F0A3F0A3F0D9
:01391500228F
:10377500908009E04420F09080B8E0706C9080B9AA
:103785007482F07F039080C6EFF07FCDA3EFF07FCA
:10379500039080C4EFF0A374CDF09080C074FFF067
:1037A500A3F0A3F0A3F09080017402F09069C21217
:1037B5001D2D000000009069C2E090804CF09069DA
:1037C500C3E090804DF09069C4E090804EF0906920
:1037D500C5E090804FF0A3E4F0A3F0A3F0A3F09030
:0937E5008024F0A3F0A3F0A3F08E
:0137EE0022B8
:103673008C288D29A907EAFDE975F018A424ACFF6D
:10368300E5F034808F82F583EDF0EBFDE975F018FA
:10369300A4FFAEF024ACFBEE34808B82F583A3ED64
:1036A300F08529828C83E0FDEF24A8FFEE3480FEB1
:1036B3008F82F583EDF08529828C83A3E08F828E40
:1036C30083A3F0852982852883A3A3E0FDE975F010
:1036D30018A424A8FFE5F03480FE8F82F583A3A30A
:1036E300EDF08529828C83A3A3A3E08F828E83A32D
:0436F300A3A3F0227B
:06345B008D2DAB07AA064F
:10346100908000E030E5079065797401F022906961
:10347100BAE0FCA3E0FDA3E0FEA3E0F5318E308DC0
:103481002F8C2EAE02AF038E838F8263A201E530B3
:10349100540744C0F58385318263A201AF2D121F09
:1034A100C7E4FCFDFEE531252DF531EE3530F53073
:1034B100ED352FF52FEC352EF52E908040E52EF0D1
:1034C100A3E52FF0A3E530F0A3E531F0908000747F
:1034D10020F0AF31AE30AD2FAC2E9069BA121D2164
:0134E10022C8
:0634E2008D28AB07AA06CD
:1034E800908002E030E5079065797403F0229069D6
:1034F800BEE0FCA3E0FDA3E0FEA3E0F52C8E2B8D3F
:103508002A8C29AE02AF038E838F8263A201E52B3A
:10351800540744D0F583852C8263A201AF28121F7B
:10352800C7E4FCFDFEE52C2528F52CEE352BF52B04
:10353800ED352AF52AEC3529F529908058E529F04A
:10354800A3E52AF0A3E52BF0A3E52CF09080027404
:1035580020F0AF2CAE2BAD2AAC299069BE121D21EC
:013568002240
:02314A008F28CC
:10314C00908001E030E5099065797402F07F0022EF
:10315C009069C2E0FCA3E0FDA3E0FEA3E0F52C8E99
:10316C002B8D2A8C2990667C63A201E52B54074495
:10317C00C8F583852C8263A2017F06121FDDE52C26
:10318C002406F52CE4352BF52BE4352AF52AE43509
:10319C0029F52990657A63A201E52B540744C8F5FB
:1031AC0083852C8263A201AF28121FDDE4FCFDFE97
:1031BC00E52C2528F52CEE352BF52BED352AF52AAB
:1031CC00EC3529F52990804CE529F0A3E52AF0A3EC
:1031DC00E52BF0A3E52CF09080017420F0AF2CAE21
:0D31EC002BAD2AAC299069C2121D21AF281D
:0131F90022B3
:102A0F009081E0E0F52805280528052805280528E8
:102A1F0005280528052805280528908010E0F52BA6
:102A2F00A3E0F52CA3E0F52DA3E0F52E9081E1E0D6
:102A3F00F52805280528052805280528052805282F
:102A4F00052805280528908014E0F52FA3E0F53020
:102A5F00A3E0F531A3E0F532E531B52D08E532B548
:102A6F002E037F0022E4F528E531540744E0F58377
:102A7F0085328263A20190637663A2017F081220E0
:102A8F000D90637863A2019062AE63A2017F06127C
:102A9F001F55906376E0F529A3E0F52AE4F5289019
:102AAF006376E0702AA3E024F8F528E53154074453
:102ABF00E0F58385328274082582F582E43583F54B
:102ACF008363A20190637663A201AF2812200DAE3B
:102ADF0029E4FCFDE532252AF532E5313EF531EDED
:102AEF003530F530EC352FF52F908014E52FF0A30E
:102AFF00E530F0A3E531F0A3E532F09080007440AB
:032B0F00F0AF28FC
:012B120022A0
:1023A3009081E6E0F5280528052805280528052855
:1023B30005280528052805280528908028E0F52B01
:1023C300A3E0F52CA3E0F52DA3E0F52E9081E7E043
:1023D300F5280528052805280528052805280528A2
:1023E30005280528052890802CE0F52FA3E0F5307B
:1023F300A3E0F531A3E0F532E4F528E531B52D0A84
:10240300E532B52E05C22002250FE531540744F00D
:10241300F58385328263A20190637663A2017F080C
:1024230012200D906376E0F529A3E0F52AE52A450D
:102433002970099080027410F07F0022906683E077
:10244300FFF46030906378E06F60030224D69066F7
:1024530084E0FF906379E06F7079906685E0FF9088
:10246300637AE06F706D906686E0FF90637BE06F48
:102473006031805F906378E0906683F0906379E0E9
:10248300906684F090637AE0906685F090637BE0D9
:10249300906686F090637CE0FFA3E090634ACFF000
:1024A300A3EFF0906376E0702AA3E024F8F528E523
:1024B30031540744F0F58385328274082582F5820E
:1024C300E43583F58363A20190637663A201AF28A9
:1024D30012200DAE29E4FCFDE532252AF532E53163
:1024E3003EF531ED3530F530EC352FF52FAF2EAE0F
:1024F3002DAD2CAC2BAB32AA31A930A82FD3121D92
:102503001040099080027410F07F002290802CE527
:102513002FF0A3E530F0A3E531F0A3E532F090808E
:06252300027440F0AF2835
:01252900228F
:10252A009081E3E0F52805280528052805280528CF
:10253A000528052805280528052890801CE0F52B84
:10254A00A3E0F52CA3E0F52DA3E0F52E9081E4E0BD
:10255A00F528052805280528052805280528052819
:10256A00052805280528908020E0F52FA3E0F530FE
:10257A00A3E0F531A3E0F532E4F528E531B52D0AFB
:10258A00E532B52E05C221022680E531540744E81A
:10259A00F58385328263A20190600463A2017F0EF3
:1025AA00122023906004E0F529A3E0F52A90600C3C
:1025BA00E0FFF4604A90667CE0FEEF6E7079A3E07B
:1025CA00FF90600DE06F706F90667EE0FF90600E86
:1025DA00E06F706390667FE0FF90600FE06F705766
:1025EA00906680E0FF906010E06F704B906681E02B
:1025FA00FF906011E06F703FE4906013F0800890E4
:10260A00601374FFF0D2D9906004E0702AA3E0242A
:10261A00F2F528E531540744E8F583853282740ED1
:10262A002582F582E43583F58363A2019060046311
:10263A00A201AF28122023AE29E4FCFDE532252AA7
:10264A00F532E5313EF531ED3530F530EC352FF523
:10265A002FAF2EAE2DAD2CAC2BAB32AA31A930A8A0
:10266A002FD3121D105006E52A45297009908001C2
:10267A007410F07F0022908020E52FF0A3E530F05F
:10268A00A3E531F0A3E532F09080017440F0AF2861
:01269A00221D
:042D04008E2D8F2E53
:102D0800908000E030E5079065797401F0229069C1
:102D1800BAE0FCA3E0FDA3E0FEA3E0F5348E338D1A
:102D2800328C31E534FFE5335407FEE42FF530EEFD
:102D380034C0F52F853082F5837423F00530E530F3
:102D48007002052F532FC7F582852F83740AF0056B
:102D580030E5307002052F532FC790633F63A201FF
:102D6800852F8385308263A2017F06121FC77406F0
:102D78002530F530E4352FF52F852D83852E826398
:102D8800A201852F8385308263A201121FABE4FC68
:102D9800FDFE9069BAE0F8A3E0F9A3E0FAA3E02FFA
:102DA800FFEE3AFEED39FDEC38FCEF2408FFE43E77
:102DB800FEE43DFDE43CFC9069BA121D219069BA1D
:102DC800E0908040F09069BBE0908041F09069BC51
:102DD800E0908042F09069BDE0908043F0908000E0
:032DE8007420F064
:012DEB0022C5
:0A2908008E2D8F2E8C2F8D308B3119
:10291200908000E030E5079065797401F0229069BB
:10292200BAE0FCA3E0FDA3E0FEA3E0F5378E368D0E
:10293200358C34E537FFE5365407FEE42FF533EEE8
:1029420034C0F532853382F5837423F00533E533E1
:10295200700205325332C7F582853283740AF0055C
:1029620033E533700205325332C790633F63A201ED
:1029720085328385338263A2017F06121FC77406E4
:102982002533F533E43532F532852D83852E826386
:10299200A20185328385338263A201121FAB8F3875
:1029A200EF2533F533E43532F532E5316017852F03
:1029B2008385308263A20185328385338263A201DB
:1029C200AF31121FC7E53824082531F531FFE4FC89
:1029D200FDFEE5372FF537EE3536F536ED3535F5B3
:1029E20035EC3534F534908040E534F0A3E535F02C
:1029F200A3E536F0A3E537F09080007420F0AF37FE
:0C2A0200AE36AD35AC349069BA121D211F
:012A0E0022A5
:062FB3008E088F098D0A53
:102FB900908000E030E5079065797401F02290690E
:102FC900BAE0FCA3E0FDA3E0FEA3E0F5108E0F8DAF
:102FD9000E8C0DE510FFE50F5407FEE42FF50CEEFE
:102FE90034C0F50B850C82F5837423F0050CE50CD0
:102FF9007002050B530BC7F582850B83EBF0050CAB
:10300900E50C7002050B530BC790633F63A2018562
:103019000B83850C8263A2017F06121FC7740625E4
:103029000CF50CE4350BF50B85088385098263A241
:1030390001850B83850C8263A201AF0A121FC77435
:1030490008250AF50AFFE4FCFDFEE5102FF510EE50
:10305900350FF50FED350EF50EEC350DF50D9080AC
:1030690040E50DF0A3E50EF0A3E50FF0A3E510F0A0
:103079009080007420F0AF10AE0FAD0EAC0D9069CA
:04308900BA121D2139
:01308D002220
:0235EE008F410B
:1035F000908000E030E5079065797401F0229069D1
:10360000BAE0FCA3E0FDA3E0FEA3E0F5458E448D07
:10361000438C42E545FFE5445407FEE42FFFEE34BA
:10362000C09062B563A201F5838F8263A201AF41AE
:10363000121FC7E4FCFDFEE5452541F545EE354486
:10364000F544ED3543F543EC3542F542908040E5D5
:1036500042F0A3E543F0A3E544F0A3E545F09080F4
:10366000007420F0AF45AE44AD43AC429069BA124D
:023670001D211A
:013672002235
:062ED2008E288F29AB05DC
:102ED800908000E030E5079065797401F0229069F0
:102EE800BAE0FCA3E0FDA3E0FEA3E0F52F8E2E8D53
:102EF8002D8C2CE52FFFE52E5407FEE42FF52BEE45
:102F080034C0F52A852B82F5837423F0052BE52B35
:102F18007002052A532AC7F582852A83EBF0052B10
:102F2800E52B7002052A90633F63A201852A8385F9
:102F38002B8263A2017F06121FC77406252BF52B6F
:102F4800E4352AF52A532AC7E528852B82852A8362
:102F5800F0052BE52B7002052A532AC7F582852A2E
:102F680083E529F0052BE52B7002052A532AC7E5CE
:102F78002F240AF52FE4352EF52EE4352DF52DE412
:102F8800352CF52C908040E52CF0A3E52DF0A3E539
:102F98002EF0A3E52FF09080007420F0AF2FAE2E16
:0A2FA800AD2DAC2C9069BA121D216A
:012FB20022FC
:0A3BE100E4FEEEC39F50030E80F8CF
:013BEB0022B7
:103B3F00A2AF9228C2AF438E2075D2028F828E839E
:0C3B4F00E0FFE4F5D2538EDFA22892AF15
:013B5B002247
:103AD300E5D220E0FBA2AF9228C2AF43D2028F828D
:103AE3008E83EDF075D25063D250A22892AFE5D207
:033AF30020E0FBD5
:013AF60022AD
:1036F700E4FDED2401FFE433FE123B3F74372DF563
:1037070082E43463F583EFF00DBD3FE6E4FDED247D
:103717007FFFE433FE123B3F742D2DF582E43461C5
:10372700F583EFF0742D2DF582E43461F583E070B5
:103737001B742D2DF582E43461F5837420F0742E0B
:103747002DF582E43461F583E4F080040DBD80BE7D
:10375700E49061ACF0FDEDFF7E00123B3F74AD2DB0
:0D376700F582E43461F583EFF00DBDFEE95D
:013774002232
:023A78008B2D94
:103A7A00A2AF9228C2AF85A22E53A2FE8E838F8256
:103A8A0005A28C838D827409122051E52D53A2FE62
:103A9A0043A22012205353A2DF852EA2A22892AF5E
:013AAA00FF1C
:013AAB0022F8
:103B5C00A2AF9228C2AF8C838D82EF12205143A268
:0C3B6C002012205353A2DFA22892AFFFCA
:013B7800222A
:023AF7008F2816
:103AF900A2AF9228C2AFE4F5838D827406122051D9
:103B0900E52843A22012205353A2DFA22892AF7FB7
:013B190001AA
:013B1A002288
:023B1B008F28F1
:103B1D00A2AF9228C2AFE4F5838D82740A122051B0
:103B2D00E52843A22012205353A2DFA22892AF7F93
:013B3D000186
:013B3E002264
:101E7A00A907E7FFA805EF93C3966008403B74FCE7
:101E8A002FFF80F00F08EF93C3966008402B74FB76
:101E9A002FFF80E00F08EF93C3966008401B74FA87
:101EAA002FFF80D00F08EF93D3966008400B74F988
:101EBA002FFF80C01F1F1F1F1FEF54FEF80303F7D9
:101ECA00E893FC08E893FD08E893FE08E893FF22EC
:101EDA0009E993C39D6008402974FB29F980F10937
:101EEA00E993C39E6008401A74FA29F980E209E965
:101EFA0093D39F6008400B74F929F980D3191919F3
:101F0A001919E9C313C313FF22740093F8ECC39899
:101F1A004024701F740193F8EDC39840197014742B
:0E1F2A000293F8EEC398400E7009740393F80A
:101F3800EFC39840037F00227F0122EDF8E6F00806
:101F4800A3DFFA22EDF8E0F608A3DFFA22E0A363A4
:101F5800A201F0A363A201DFF475A2002263A2012B
:101F6800F0A363A20122E0A363A201F0A363A2018C
:101F7800E0A363A201F0A363A201E463A201F0A3BA
:101F880063A201DFE175A20022E0A363A2016DFE56
:101F9800936CFDEE058393FC158363A201DFEA755C
:101FA800A200227F00E493A363A201F00F600CA3B8
:101FB800E583C2E3F58363A20180EA75A20022E00B
:101FC800A363A201F0A3E583C2E3F58363A201DF63
:101FD800EE75A20022E0A363A201F0A3E583C2E4A8
:101FE800D2E3F58363A201DFEC75A20022E0A363CC
:101FF800A201F0A3E58344F8C2E5F58363A201DFFB
:10200800EC75A20022E583C2E3F583E0A363A20195
:10201800F0A363A201DFEE75A20022E583C2E4D239
:0A202800E3F583E0A363A201F0A337
:1020320063A201DFEC75A20022E58344F8F583E098
:10204200A363A201F0A363A201DFEE75A20022F94D
:1020520022C002C004C00612FFF0D006D004D00293
:01206200225B
:1033DB000208DFE493A3F8E493A34003F68001F221
:1033EB0008DFF48029E493A3F85407240CC8C333F3
:1033FB00C4540F4420C8834004F456800146F6DFC2
:10340B00E4800B0102040810204080903B79E47E9D
:10341B00019360BCA3FF543F30E509541FFEE493B6
:10342B00A360010ECF54C025E060A840B8E493A37D
:10343B00FAE493A3F8E493A3C8C582C8CAC583CAA8
:10344B00F0A3C8C582C8CAC583CADFE9DEE780BE60
:013B94000030
:101C0900BB010689828A83E0225002E722BBFE02D9
:091C1900E32289828A83E493220C
:101C2200BB010689828A83F0225002F722BBFE01A1
:021C3200F3229B
:101C340075F008758200EF2FFFEE33FECD33CDCC67
:101C440033CCC58233C5829BED9AEC99E5829840EA
:101C54000CF582EE9BFEED9AFDEC99FC0FD5F0D6C7
:101C6400E4CEFBE4CDFAE4CCF9A88222B800C1B9F1
:101C74000059BA002DEC8BF084CFCECDFCE5F0CB2F
:101C8400F97818EF2FFFEE33FEED33FDEC33FCEB68
:101C940033FB10D703994004EB99FB0FD8E5E4F923
:101CA400FA227818EF2FFFEE33FEED33FDEC33FC10
:101CB400C933C910D7059BE99A4007EC9BFCE99A04
:101CC400F90FD8E0E4C9FAE4CCFB2275F010EF2F49
:101CD400FFEE33FEED33FDCC33CCC833C810D70749
:101CE4009BEC9AE899400AED9BFDEC9AFCE899F884
:0E1CF4000FD5F0DAE4CDFBE4CCFAE4C8F92217
:0E1D0200C3E49FFFE49EFEE49DFDE49CFC22F2
:101D1000EB9FF5F0EA9E42F0E99D42F0E89C45F029
:011D200022A0
:0C1D2100ECF0A3EDF0A3EEF0A3EFF02235
:101D2D00A8828583F0D083D082121D44121D4412E7
:101D3D001D44121D44E473E493A3C583C5F0C5830C
:101D4D00C8C582C8F0A3C583C5F0C583C8C582C800
:011D5D002263
:1018AD00E53C2430F8E6053C22782D302F027830C7
:1018BD00E475F001121DDA021C092028EB7F2ED2EF
:1018CD00288018EF540F2490D43440D4FF302C0BC3
:1018DD00EF24BFB41A0050032461FFE53D600215EB
:1018ED003D0540E5407002053F302F0D782DE47524
:1018FD00F001121DDAEF021C220239C17403D22F3E
:10190D008003E4C22FF53C8B2D8A2E892FE4F53D03
:10191D00F53FF540E53D60077F201218E880F5752D
:10192D003EFFC229C228C22AC22BC22DC22EC230EE
:10193D001218B6FF700D302F057F001218F9AF4049
:10194D00AE3F22B4255FC2D5C22C1218B6FF24D0EB
:10195D00B40A00501A75F00A783D30D50508B6FF67
:10196D000106C6A426F620D5047002D22B80D924F8
:10197D00CFB41A00EF5004C2E5D22C021AF9D229C5
:10198D0080C6D22880C0D22A80BCD2D580BAD22DB2
:10199D0080B47F201218E8202A077401B53D00405D
:1019AD00F11218ADFF1218E8021921D230D22E8093
:1019BD00951218ADFB1218ADFA1218ADF94A4B700D
:1019CD000679CA7A1B7BFF202A2EE53D602A7E0010
:1019DD008E82758300121D5E60060EEE653E70F000
:1019ED00C2D5EBC0E0EAC0E0E9C0E0EE121B40D08A
:1019FD00E0F9D0E0FAD0E0FB121C09FF60AAEBC0C1
:101A0D00E0EAC0E0E9C0E01218E8D0E02401F9D026
:101A1D00E03400FAD0E0FBE53E0460DCD53ED98031
:101A2D00877BFF7A1B793CD22A809C7910800279C2
:101A3D0008C22EC2308008D2D5790A8004790AC234
:101A4D00D5E53E047002F53EE4FAFDFEFF1218AD39
:101A5D00FC7B082029131218ADFD7B1030280A12CB
:101A6D0018ADFE1218ADFF7B20EC3382D592D55008
:101A7D0013C3E43028069FFFE49EFEE42029039D56
:101A8D00FDE49CFCE4CBF8C229EC700CCFCECDCCA0
:101A9D00E824F8F870F38017C3EF33FFEE33FEED53
:101AAD0033FDEC33FCEB33FB994002FB0FD8E9EB34
:101ABD00302905F8D0E0C448B229C0E00AEC4D4EFB
:101ACD004F78207B0070C2EAB53E0040BCC0E012EA
:101ADD001B42D0F0D0E0202904C4C0E0C4B229C01C
:101AED00F01218D1D0F0D5F0EB021921121E3919D0
:101AFD00BE531A3858198F4C198B421A3C4F1A4441
:0F1B0D00441A444919A4431A4A551A2E461A2E4F
:101B1C00451A2E471BEA5019932D19972E19BA2BDB
:101B2C00199B2319B8201BD32A195348000019B24A
:101B3C003F3F3F00790AA2D5202B14302D09B91054
:101B4C00020404B9080104A2D5202E02500104207D
:101B5C002A68922AB53D005034C0E07F20302B1902
:101B6C007F30A22A722E722D500F121B99C22AC2DC
:101B7C002EC22DC2307F30800F302D03E9C0E01211
:101B8C0018E8302D03D0E0F9D0E0B53DCC302D175E
:101B9C007F30B9100C1218E87F58302C077F7880F2
:101BAC0003B908031218E8302A057F2D0218E87FC4
:101BBC00202030F87F2B202EF322922A80CF286E03
:101BCC00756C6C2900D2291218AD3029F8C229780D
:101BDC003D30D50108F60219532D504349581218BF
:101BEC00AD2403B405004001E4901BE5931218D911
:0D1BFC00743A1218D9D22B753D04021A3824
:102063008B288A29892AE4F534F533F532F531F5DD
:102073002FF530E52C452D452B6012EBC0E0EAC06F
:10208300E0E9C0E0AB2BAA2CA92D121DEAAB280571
:102093002AE52AAA297002052914F9121C09F53523
:1020A300C394094007E535D3940D40E1E535642039
:1020B30060DBE535B42D054330038016E535B42BDD
:1020C30005433001800C74FF252AF52A74FF352956
:1020D300F529E52E60046410703FAB28AA29A92ACC
:1020E300121C0964306009E52E702E752E0A8029B2
:1020F300900001121D5EFF64786004EFB45813432F
:102103003001752E107402252AF52AE43529F529A4
:102113008007E52E7003752E08AB28052AE52AAA49
:10212300297002052914F9121C09F535C39461407D
:102133000AE535D3947A50035335DF74D02535F54A
:1021430035C3940A400CE5359411406D74F9253577
:10215300F535E535D3952E50604330018534398507
:102163003338853237853136AF2E7E00E4FCFDAB44
:1021730034AA33A932A831121D8BC8ECC8C9EDC9E2
:10218300CAEECACBEFCBE4FCFDFEEB2535F534EE0E
:102193003AF533ED39F532EC38F531AF34AE33ADD2
:1021A30032FCAB39AA38A937A836D3121D10500315
:1021B30002211C43300402211CE53020E003E480AB
:1021C3002DE52C452D452B601EAB28E52A24FFF970
:1021D300E52934FFFAEBC0E0EAC0E0E9C0E0AB2B4D
:1021E300AA2CA92D121DEAE53030E20774FFFFFE89
:1021F300FDFC22E530AF34AE33AD32AC3130E10318
:04220300021D022294
:101D5E00BB010CE58229F582E5833AF583E022503A
:101D6E0006E92582F8E622BBFE06E92582F8E22284
:0D1D7E00E58229F582E5833AF583E493229E
:101D8B00E88FF0A4CC8BF0A42CFCE98EF0A42CFCF7
:101D9B008AF0EDA42CFCEA8EF0A4CDA8F08BF0A475
:101DAB002DCC3825F0FDE98FF0A42CCD35F0FCEBD4
:101DBB008EF0A4FEA9F0EB8FF0A4CFC5F02ECD3999
:0F1DCB00FEE43CFCEAA42DCE35F0FDE43CFC2206
:101DDA00FAE6FB0808E6F925F0F618E6CA3AF6220A
:101DEA00BB011A89828A83D0F0D0E0F8D0E0F9D01A
:101DFA00E0FAD0E0FBE8C0E0C0F0021E685016E945
:101E0A00F8D083D082D0E0F9D0E0FAD0E0FBC082EB
:101E1A00C083021E5FBBFE16E9F8D083D082D0E0F1
:0F1E2A00F9D0E0FAD0E0FBC082C083021E712223
:101E3900D083D082F8E4937012740193700DA3A338
:101E490093F8740193F5828883E47374029368604C
:061E5900EFA3A3A380DF4C
:091E5F00EBF608EAF608E9F622A8
:091E6800EBF0A3EAF0A3E9F0227B
:091E7100EBF208EAF208E9F222A2
:00000001FF
